:030000000219FDE5
:03000B000200AA46
:03002B0002015F70
:03005B000202E7B7
:030073000202CDB9
:1000800002030406080C10182030406080040608A3
:100090000C10182030406080A0C000070F1F3F0DDB
:1000A0000D04050D050205030302C2AFC0D0C0E078
:1000B000206217E5256002E473E525F4F58A758B67
:1000C00000D262D0E0D0D0D2AF3285268AC262E5BB
:1000D00026F4602F758B00D0E0D0D0D297D295D285
:1000E00093D2AF32D297D295D293206E0C2066096C
:1000F0007405D5E0FDE57E4290758B00D0E0D0D050
:10010000D2AF32758A00C28DD26201F901B930686E
:1001100005206602C29701B9306805206602C293C5
:1001200001B9306805206602C29501B9C2963068EF
:100130000A2066077419D5E0FDC29701B9C2923052
:10014000680A2066077419D5E0FDC29301B9C2940C
:1001500030680A2066077419D5E0FDC29501B9C25E
:10016000AFC2AD53E6EFC0D0C0E0D2D3D2AFC2CE63
:10017000E52A6007207449152A21C07800790020FB
:10018000742EE580307E01F430E50278FF53DACF3B
:10019000207E0343DA20307E0343DA10C2D8C271D6
:1001A000E580307E01F430E50279FFC3E89970CB39
:1001B000306103752A18207403752A18885FD2707D
:1001C00020740DE52B6004152B21D043DA01C2D831
:1001D000207002412EA85F206102C270207436791F
:1001E00082B70431C3E894F0400374F0F8E8C454D3
:1001F0000F28F87984B703024115C313C31387216D
:10020000200802C313200A06C3C898F8411528F82D
:10021000500374FFF88822E52D54066011E533C3BE
:1002200013C31324062522F52250037522FF78827A
:10023000B6044E852224A824C3E52495644002A870
:1002400064C3E895664002A8668825E569700241A6
:100250007FC3E8AA699A5003E8FAE4F9EAC333FBDA
:10026000E56BF45B29400D256AF8E56A6002156AC2
:10027000400B417F0AC3E56A9A5002056A78FF88FD
:1002800026C3E52594404002D26420CF0AD0E0D0B6
:10029000D043E610D2AD32C2CF053A7801E52A60EC
:1002A00005307402152AC3E55F94014005756200AC
:1002B00041C3756300756C00E5622401F56250036B
:1002C0007562FFD0E0D0D043E610D2AD32C2AFC0ED
:1002D000D053E67FC2607591008556948557957519
:1002E0009104D0D0D2AF32C2AF53E6EFC2ADC0D08E
:1002F000C0E0C0F0D2D3D2AFA8FBA9FCC2D8307105
:1003000002614E53DACF207E0343DA10307E03437E
:10031000DA20D271E580307E01F420E50261258883
:10032000278928A17B53DACF207E0343DA20307E51
:100330000343DA10C2D8C271307402A1677800E5B5
:1003400080307E01F430E502A167885FA14F53DA67
:10035000CF207E0343DA20307E0343DA10C27120BF
:100360006102812753DACF207E0343DA10307E0307
:1003700043DA20C2D8D271885A895BC3E89558F80D
:10038000E99559F97B007E087A00C3E8948CE994DA
:10039000005005755E008119882178A2E6A82160C9
:1003A00055C3E894C8E994005008E4D2E4FB7A0A03
:1003B00061F4C3E89468E994015008E4D2E3FB7A5D
:1003C0000F61F4C3E894D0E994025008E4D2E2FB50
:1003D0007A1E61F4C3E894A0E994055008E4D2E1E0
:1003E000FB7A3C61F4C3E89498E994085008E4D29D
:1003F000E0FB7A787E00C3E8955CFCE9955DFD3012
:10040000E70AECF42401FCEDF43400FD755E00C352
:10041000EC9AED9E5003755E01885C895D855A58A3
:10042000855B597802A14FC3E89527F8E99528F92B
:10043000307C02A133307B02A133307A02A12C2020
:100440007502814AE9FDE8FC8169E9C313F9E81303
:10045000F8307902A12CE9C313F9E813F8307802D7
:10046000A12CE9C313FDE813FC20612CC3EC941C00
:0E047000ED940240028180ED701EC3EC94C832
:10047E0050180529E52970021529C3E529940A505B
:10048E0002A167755F00D270A167E5296002152988
:10049E007888E6F97400207F087896B90302789E72
:1004AE00E624FAFEE43400FFC3EC9EFCED9FFD92C1
:1004BE0008B90310A2085007207609D27681D230EF
:1004CE007602C276A2085016B9030DECF42401FC94
:1004DE00EDF43400FD0204EC78007900A133B90389
:1004EE0015EC33FCED33FDC3EC940AFCED9400FDEA
:1004FE0050047C007D00C3EC94FFED940040067820
:10050E00FF7900A133EC8575F0A4C5F0A2F733F89E
:10051E007900400302054F78FF790002054FE9C3C9
:10052E0013F9E813F8307C0EE9600278FFC3E81384
:10053E0038F8E43400F9C3E894FFE99400400278F7
:10054E00FF885FD270206102A167741FF4552F4B94
:10055E00F52FC274EB7002D274752A1830740375BD
:10056E002A0A306102A17B20740353DAFE20740341
:10057E00752B06D0F0D0E0D0D0D2AD43E610327954
:10058E00010205AB79030205AB790A0205AB791EB0
:10059E000205AB79640205AB79C80205AB7817E4A6
:1005AE00D5E0FDD8FAD9F6227A147B780205D27AF4
:1005BE00107B8C0205D27A0D7BB40205D27A0B7BAE
:1005CE00C80205D27902B27DE4C292D5E0FDC29393
:1005DE00D5E0FDD293D5E0FDD292D5E0FDC297E5F0
:1005EE0076D5E0FDD2977496D5E0FDD9D9EAF8D547
:1005FE00E0FDD8FBDBCEC29222C37C007D0075F0FD
:10060E000005F0EA33FAEB33FB50F6EB13FBEA137B
:10061E00FAC3E9FFE8FEE89AF8E99BF95004EFF90E
:10062E00EEF8B3EC33FCED33FDD5F0DFEDF9ECF87D
:10063E0022E889F08A20D2D4F8A9F07B0030F70B9B
:10064E007BFFF42401F8E9F43400F9E88520F0A4E6
:10065E00ADF0F8E98520F0A4AFF0FEED2EF97400B0
:10066E003FFA7C04C3EA13FAE913F9E813F8DCF451
:10067E008BF030F70AE8F42401F8E9F43400F9E8D5
:10068E0089F0C2D4F8A9F0227882B604030206F1EA
:10069E00C3E55F940140030206BB852224E4F545C1
:1006AE00F546F547F548F549C26D0206F17882E642
:1006BE00FCD26DE522F523783879C7AA40AB41C349
:1006CE00EB13FBEA13FAEC146013C3EB13FBEA1300
:1006DE00FAEC14146007C3EB13FBEA13FAD1078884
:1006EE0045894622C3E5459523F8E5469400F95021
:1006FE000CC3E89480E994FF4016020722C3E894E5
:10070E007FE994005003020722787F7900020722C6
:10071E00788079FF884A894B22E54A2547F8E54BD0
:10072E003548F9854B20E4300701F43549FA30E7B6
:10073E0009C3EA94F04015020760C3EA940F500310
:10074E0002076078FF79FF7A0F0207607800790060
:10075E007AF0C3E5249564500AC374019524500BB6
:10076E0002077EE54B20E70E02077EE54B30E706DB
:10077E00884789488A492278A4E6FAC3E54A33F8BD
:10078E00E54B33F9D13FE930E70BC3E89480E994A8
:10079E00FF4013E1B8C3E8947FE994005002E1B83A
:1007AE00787F7900E1B8788079FFE820E715C3E516
:1007BE002398F84009C3E8940140030207DF78014B
:1007CE000207DFE8F424012523F840030207DF784F
:1007DE00FF884C2278A5E6FAA848A949D13FE9300E
:1007EE00E70CC3E89401E994FF4016020813C3E82E
:1007FE0094FFE99400500302081378FF7900020871
:10080E0013780179FFE920E715C3E54C98F8400904
:10081E00C3E89401400302083A780102083AE8F46A
:10082E002401254CF8400302083A78FF88242278E8
:10083E00FFC26420693D206A12D264C3E541940A66
:10084E004009C3E52594405002C26479A1E76023B4
:10085E00E541601F74FF8541F0848539F0306A03ED
:0F086E0075F005A4F8C5F0600278FFC3E8956740
:10087D005002A867886622C3E5409440E541940183
:10088D00E5665003140195046002F5662202089D89
:10089D002275E890227883E6FFE5E820ECF7A8BD05
:1008AD00A9BE0573C3E57394084052757300E9FA48
:1008BD0079A0E76044EA7007E574601B0208D8C3AD
:1008CD00E895746010E5745006600C140208E40499
:1008DD0060F90208E4E574F574C3946D401B75640A
:1008ED00C0C394044013756480C39404400B7564B5
:1008FD0040C39404400375640075BB0822E564246D
:10090D0010500274FFF5647982B704022131C3A837
:10091D0064E524985002A824C3E895664002A866B1
:10092D0088258826E573B4070375BB1022743279C8
:10093D00A687F0A4C5F0A2F733F8C3E8956440028A
:10094D00A864882288248825882688672275400017
:10095D007541F022C2AF75C820A8CCA9CDAA3A30F6
:10096D00CF010A75C824D2AFAB3BAC3C883B893C68
:10097D00C3E89BF8E99C206908F9306702417621AC
:10098D00D3AD3D8A3DF9EA9DFA600478FF79FFAE5B
:10099D003EAF3F8B3E8C3FC3EC9FFCC3E99CF542C1
:1009AD00A83BA93CC3E89EF8E99FF9C3E54113FBB9
:1009BD00E54013FAE82AF540E93BF541500675404C
:1009CD00FF7541FF411DAA40AB41AC40AD417E04D6
:1009DD007F02C3EB940440021E1FC3EB9408400238
:1009ED001E1FC3ED13FDEC13FCDEF7C3EA9CFAEBFF
:1009FD009DFBEF6009C3E913F9E813F8DFF7EA2867
:100A0D00FAEB39FB8A408B4150067BFF8B408B41C3
:100A1D00C3EB94025002D2673069047F03414878DA
:100A2D0092E6FFC3E537948240110FC3E53794A0DA
:100A3D0040010FC3EF940640027F057E07E541C4D8
:100A4D00540FF9E541C454F0F8E540C4540F28F8AB
:100A5D00C3E89EFAE99400FB4009C3EA9402EB94C3
:100A6D000050047A02E4FB41C2AA40AB41EBC4FE44
:100A7D00EAC4540F4EFCC3EA9CFAEB9400FBC3E8A6
:100A8D0013C313F8EA28FAEB3400FB8A408B41C3F9
:100A9D00EB94024002C2677807EBC4FE7B00EAC408
:100AAD00540F4EFAC3EA98FA4005C3940250027AE5
:100ABD00027892E6FF30600241C285525685535747
:100ACD00D26043E680C3E49AF8E49BF93067026193
:100ADD005CE8FAE9FBD3E913FDE813FC885289536E
:100AED00C3EF94036038EF20E00DE82CF8E93DF9F1
:100AFD00ECFAEDFB020B17E828F8E939F9C3E82405
:100B0D0002F8E93400F97AFE7BFFC3EF9403400E3F
:100B1D008A548B55884E894F8C508D5161908854D5
:100B2D0089558A4E8B4F8C508D51306920C3E533DA
:100B3D0094034019E542A2E713F8E555F424013872
:100B4D00400B20E7087554FFF42401F5556190E83A
:100B5D00FAD3E813FC8852C3EF94036020EF20E032
:100B6D0007E82CF8ECFA617CE8282402F87AFEC339
:100B7D00EF940340088A54884E8C50619088548AB3
:100B8D004E8C50E56BC3335002646BF56B306002D5
:100B9D00619A753402D26043E680E52D54066026D5
:100BAD00A840A941C3E913F9E813F8C2AF53E67F92
:100BBD00759100C3E498F594E499F595759104D277
:100BCD006043E680D2AF22D26575440075200030B7
:100BDD006B03752040020BF3D26575440075204000
:100BED00306B03752000D2AF7801206722E52D54BC
:100BFD00066002C265C3E541940540137802940571
:100C0D0040087803940540027806306902780A207E
:100C1D006019E544601530690AC3E5339403400358
:100C2D00D53406D2AFD26C81C471A2D2AF0000C24E
:100C3D00AF206726E541C3FB940F40027B0FEB24E9
:100C4D000530730123306A02742820620123F930C4
:100C5D0069027982E58BC39940B50544E59B544003
:0F0C6D00B5200281AE30690A08C3E8940A40013D
:100C7C0008811C20650261F3C26553E67F75910003
:100C8C003067107594007595FE759104D26043E63B
:100C9C008061F3AE40AF41C3E49EF594E49FF595BB
:100CAC008195C3E5339402500261F330650261F320
:100CBC00D80281C2811CC26C53E67F7591008554A9
:100CCC0094855595759104854E56854F57D2604342
:100CDC00E680D2AFE52D54066008206A0205330287
:100CEC000CFE306C0D206B0A2065071581158102F6
:100CFC0015642278003064053065027801E537759B
:100D0C00F007A4F9E5F028F5F0E9A2F013A2F1132D
:100D1C00A2F213F537C394785003753778C3E537CF
:100D2C0095384008D266D297D295D293306002A102
:100D3C0038855056855157D26043E68022207D116C
:100D4C00C2AF754302C292D296D2AF759F13020FF7
:100D5C0018C2AF754302C292D294D2AF759F1302E0
:100D6C000F18307243207D20C2AF75430390013DB4
:100D7C00757E04D295C294306204C293A18CD29237
:100D8C00D2AF759F10020F18C2AF75430390013D8F
:100D9C00757E04D297C296306204C293A1ACD292F3
:100DAC00D2AF759F11020F18207D17C2AF75430388
:100DBC00900118D295306202C293D2AF759F100287
:100DCC000F18C2AF754303900118D297306202C25C
:100DDC0093D2AF759F11020F18207D11C2AF7543CE
:100DEC0004C296D294D2AF759F11020F18C2AF7580
:100DFC004304C294D296D2AF759F10020F18307272
:100E0C0043207D20C2AF75430590012C757E40D2E6
:100E1C0093C292306204C297C128D296D2AF759F0A
:100E2C0013020F18C2AF75430590014E757E10D298
:100E3C0093C292306204C295C148D294D2AF759FCE
:100E4C0013020F18207D17C2AF75430590010ED207
:100E5C0093306202C297D2AF759F13020F18C2AFC4
:100E6C00754305900122D2933062EBC295D2AF75D7
:100E7C009F13020F18207D11C2AF754306C294D286
:100E8C0092D2AF759F10020F18C2AF754306C2966F
:100E9C00D292D2AF759F11020F18307242207D2072
:100EAC00C2AF75430190014E757E10D297C2963039
:100EBC006204C295C1C4D294D2AF759F11020F18AF
:100ECC00C2AF75430190012C757E40D295C294300F
:100EDC006204C297C1E4D296D2AF759F10E118207C
:100EEC007D16C2AF754301900122D297306202C2C7
:100EFC0095D2AF759F11E118C2AF75430190010EE9
:100F0C00D295306202C297D2AF759F10C266229002
:100F1C00010C757E00D297D295D293C296C294C220
:100F2C0092C26222788076090876090876040876DF
:100F3C00FF0876030876FF08760908760108760123
:100F4C00087601788C76010876FF0876FF0876FF24
:100F5C000876FF0876FF0876030876FF0876FF0808
:100F6C0076FF0876250876D008762808765008761D
:100F7C00040876FF08760208760008767A0876FF71
:100F8C00087601087601087600087603227887E651
:100F9C00FFC2727888E6C394036008C27DE630E134
:100FAC0002D27DC27E7889E630E102D27EC3EF9414
:100FBC00026008758E01D273020FCC758E00C2735D
:100FCC00227880E6149000809378A4F67881E61459
:100FDC009000809378A5F67886E61490008D93782F
:100FEC00A6F6789CE67538FF75390CB40206753890
:100FFC00A075390AB4030675388275390578A3E6ED
:10100C001490009A93F569120F1B22227896E6FA37
:10101C007897E6FB7888E6B40305C3EB940EFB30B7
:10102C007F047A007BFFC3EB9AFCC3948250027C52
:10103C00827575000575EC8575F0A4C3E5F0947D9B
:10104C0040F222D27F111812059C7A007B007C1092
:10105C00120592E55F2AFA74003BFBDCF37C04C3B7
:0E106C00EB13FBEA13FADCF7FEC27F11182229
:10107A00E5EF20E6037520000520903FFFE52014E8
:10108A006006901DFF1460009304600375EF12530D
:10109A00D9BF7581C043FF8012058D75EF0243B237
:1010AA0003E5B3240420E70DF521E5E320E00685F6
:1010BA0021B343E301120F1B7580FF75A40075F17C
:1010CA00B275D4DF7590A975A5FC75F2FE75D501C8
:1010DA0075A60175E241E4F8F6D8FD756B01120FA9
:1010EA00301215A678988676753001C2AF1205A619
:1010FA001205B612059C1205BD12059C1205C412F2
:10110A00059CC2AF78FA79FA308507D9FBD8F7027D
:10111A001C00120F99120FCD1117111878988676A4
:10112A00120F1B75885075891275C824759104753C
:10113A00D84075A82275B80275E690759B80759D92
:10114A000075D10E75BC5875BB0875BA1175E88063
:10115A0012058DD2AF12089A53DACF207E0343DAF2
:10116A0020307E0343DA1043DA01C2D8C271120575
:10117A00A6D2617B037A0CE55E70077A0CDB030268
:10118A00110C12059C20700302110CC270E55FC39A
:10119A00940240E1E52F541F856160F561B560D581
:1011AA00DAD5C26153DACF207E0343DA20307E03D8
:1011BA0043DA10C2D8C27178A2E67008D274E52F59
:1011CA0054E0F52FC2757529001205A1307409C3C0
:1011DA00E529940A4002D275120592780230740207
:1011EA007800C3E55F9840F0C2AF1205B61205B6A3
:1011FA001205B6D2AF1205A6754D007888E6B4037B
:10120A000241E3120592788CE6C39401500302125C
:10121A00E3E530C3940150030212E3207435C3E5B9
:10122A005F94FF50030212E3C2AF1205CBD2AF1292
:10123A0005A1C3E55F940150EFC2AF1205B61205CE
:10124A00971205B6D2AF1205A1C3E55F94FF40E934
:10125A0002174E7F02D27F11181205A1C2AFC27FB8
:10126A001118AE5FC3E55F947FD2AF407612058D49
:10127A00C2AF1205CBD2AFDFDC114FC3EE940578B3
:10128A0097F61205A61215E81216D17F0AD27F1117
:10129A00181205A1C2AFC27F1118AE5FC3E55F94F1
:1012AA007FD2AF50E612058DC2AF1205B61205976E
:1012BA001205B6D2AFDFD6114FEE24057896F61294
:1012CA0005A61215E81217001205A11118C3E55F49
:1012DA0094FF5002412502174EC3E55F954D400326
:1012EA00855F4D1205A178017988E7B40302780574
:1012FA00C3E55F9840024105C2AF1205CB1205CB88
:10130A001205CBD2AF1205A6753000E4F531F532DD
:10131A000531E531F470390532789AE678191460A6
:10132A0012783214600D787D14600878FA1460031C
:10133A00753200C3E53298401715327531B4789981
:10134A008676C2AF1205CBD2AF789886761205A1FF
:10135A00120597E52A7005307402210C7801207471
:10136A00027806C3E55F9840A77888E6C3940360CD
:10137A00031205A1E52A700302110CC2AF120F1B5A
:10138A00E4F522F523F524F525F526F56AD2AF789A
:10139A0085E6C333F568E4F545F546F547F548F5BE
:1013AA0049F573F52CF52DF53775730875BB1012D1
:1013BA00058D12089EE5E820ECFBA8BDA9BEE970E0
:1013CA0001F888741208A275730875BB107887E64D
:1013DA00FE7602120F997887EEF6C2AF7564FF1295
:1013EA00093A852264852265852266D2AF75220173
:1013FA0075240175250175260185636C756D017863
:10140A0088E6B40307C27D307602D27DD268D269FB
:10141A00753300120E81120EA612095A12096112B0
:10142A00095A12096112095A021442C2AF120F99DB
:10143A00D2AF75730075BB08120BE5120696120C33
:10144A00FF120D49120961120BD4306D031206F214
:10145A0020670312083D306703120884120CFF123A
:0E146A000D6E120961120BE5306D031207279B
:10147800120CFF120DE5120961120BD4306D031224
:101488000785120CFF120E0A120961120BE5306D66
:10149800031207E2120CFF120E8112096112089E54
:1014A800120BD4120CFF120EA61208A212096130F8
:1014B8006935206B3285676485676585636C756DF2
:1014C8000179187A0CC3E53399400FC269D26A8A48
:1014D800358567648567660214EFC3E55F9401404C
:1014E8000302144202156C306A1B206B18E5351490
:1014F8007004C26A8135F535C3E55F940140030283
:10150800144202156C753600C3E56278FA98505497
:10151800307404E52A604D7888E6B40317207D0509
:10152800207607A13C307602A13C206B07D26B8560
:101538006764818178F0306B058567647820C3E53E
:10154800419850028142306B1BC26BC27D307602DB
:10155800D27DD26A75351285676481420536E55FAA
:101568006002A16F753600C2AF120F1B7887E6FEC6
:101578007602120F997887EEF6E4F522F523F52422
:10158800F525F526F568C268D2AF12058D120F1B36
:10159800307409C3E53694054002210C6115901A90
:1015A8000D782012162AE520B4550CA312162AE548
:1015B80020B4AA030215C8120F301215E80215E765
:1015C800901A0378807B0A12162AA308DBF9901A6E
:1015D8000F788C7B1812162AA308DBF9901A272299
:1015E800C2AF121669121643901A00740E12162F03
:1015F800A3740412162FA3741412162F901A0378CA
:10160800807B0A12162EA308DBF9901A0F788C7BC0
:101618001812162EA308DBF912167C12165A901A05
:101628002722E493F622E6438F01538FFD75EF02DC
:1016380075B7A575B7F1F0538FFE22438F02438F1C
:101648000175EF0275B7A575B7F1901A0DF0538FB4
:10165800FC22901A0D7455D12F901A0E74AAD12F0E
:10166800227A3079D07820901A40D12AE520F709DB
:10167800A3DAF7227A3079D0901A40E7D12F09A35C
:10168800DAF922AB77A878BB01027980BB0202792C
:1016980081BB03027982BB04027984BB0502798687
:1016A800BB06027992BB07027987BB080279A3BB04
:1016B8000902799CBB0A027988BB0B027989E8F791
:1016C800227C051205A6DCFB22C2AF1205B6120564
:1016D800BD1205C41205CB1205971205B61205BD39
:1016E8001205C41205CB1205971205B61205BD12D4
:1016F80005C41205CBD2AF22C2AF1205CB1205C466
:101708001205BD1205B61205971205CB1205C412B3
:1017180005BD1205B61205971205CB1205C41205B0
:10172800BD1205B6D2AF22AE77AF78C2AF1205B6FA
:101738001205B61205B6120597DEF21205CB120590
:1017480097DFF8D2AF22D1D1D1C9D1C97577017548
:101758007801757900F12F7C05AD5F1205A6C3ED00
:10176800955F70F5C3E55F9401400AC3E55F94FF98
:10177800403202178AD18BB1E8D1D1C2AF75EF12CE
:10178800D1C9DCD50579C3E5799403500280C6D167
:10179800C90578E5771490009F93F808C3E5789811
:1017A800500280AED1C9D1C90577C3E577940C50F2
:0F17B80002809C120F30B1E8C2AF75EF12D1C999
:0319FD0002107A5B
:101A00000E0414090904FF03FF0901010155AA018D
:101A1000FFFFFFFFFF03FFFFFF25D0285004FF0259
:081A2000007AFF01010003FF41
:101A4000235475726E69677933304123202020203A
:101A500023424C48454C4923463333302320202031
:101A60002020202020202020202020202020202076
:101C0000C2AFC2D353D9BF7581C043B20343FF8073
:101C1000752438752503B1C975EF0275E24043F1AB
:101C20002053A4DF75D400D2857DFA780379E67C51
:101C300010752200752300901DD67B0675249875BB
:101C400025013085028142208508D8FBD9F9DCF7CF
:101C500081B4308508D8FBD9F9DCF781B4B189E4C7
:101C600093A3C39A6004DDC381B4DBDBB17B600264
:101C7000812B7B08E493FAA3B15CDBF87A30B15C8A
:101C8000752200752300B17BEAFCEBFDC3ED94FEE9
:101C9000400EB17B8A278B28ED30E0048A828B834B
:101CA000B17B7AC270D8C3ED94FE601350CEBD00F4
:101CB00025EC60097520007521FF0200008100A855
:101CC00027A9280809D804D90281D3B17FEA89AAB3
:101CD000F281C50D81A0C3ED94035049EDA2E092BD
:101CE000007AC5C3E5829400E583941C50902000DF
:101CF00010438F02438F0175B7A575B7F1F030001F
:101D00001FA827A9280809438F01538FFDD804D99C
:101D100002A12089AAE275B7A575B7F1F0A3A10DBC
:101D2000538FFC817C7AC1BD030CE493A3FAB140CC
:101D3000DCF8B138817C817EAA22AB23B15CEBFA5E
:101D4000EA6222752608C3E52313F523E52213F57D
:101D50002250066323A0632201D526EAB1C9B1C986
:101D600075260AEAF4200102D285300102C285B14B
:101D7000C9C3134002C201D526EB22B17FEAFB2082
:101D80008502A17F308502A184752608AE24AF2587
:101D9000C3EF13FFEE13FEB1CDB1C9C3EA13308513
:101DA000024480FA30E703632201C3E52313F523DD
:101DB000E52213F52250066323A0632201D526D91C
:101DC000E52265236523F52222AE24AF250E0FDE22
:101DD000FEDFFCD20122424C48656C693437316326
:041DE000F3300601D5
:00000001FF
